:100000000AC022C021C020C01FC01EC01DC01CC00D
:100010001BC01AC019C011241FBECFEDCDBF10E008
:10002000A0E6B0E0E4E3F7E003C0C89531960D9296
:10003000A036B107D1F710E0A0E6B0E001C01D92F4
:10004000A33AB107E1F7D4C0DBCF81E44DD286E516
:100050004BD282E549D280E247D289E445D283E59A
:1000600043D280E541D208950F931F93CF93182F69
:100070003FD2082F3DD2C82F802FF0D18C2FEED148
:1000800037D2ECD1112369F033D20C3A59F4C03A8B
:1000900011F0C03E11F48FEF05C0C83A19F489E49D
:1000A00001C0812FDBD120D285E090E06CD18DE0C2
:1000B0001BD2CF911F910F910895DF92EF92FF9283
:1000C0000F931F93CF93DF93E82EF92ED62E20E0C7
:1000D00030E0D32FC22FC05ADF4F022F132F0F5FF4
:1000E0001F4F2E153F0510F403D201C08FEF8883F8
:1000F000312F202F0034110560F320E030E0809193
:10010000A2008A3319F0932F822F3CC00091A000E7
:100110001091A10086E4D81699F5CFE5D0E080E4EF
:100120009DD18091A1009AD18091A00097D1219674
:10013000899194D188E492D18091A1008FD180914E
:10014000A0008CD188818AD18091A0009091A100DB
:1001500001969093A1008093A0008EEF9FEFE80E90
:10016000F91EE114F104D9F68CE478D1812F992796
:1001700075D1802F73D180E071D185E090E003D1FB
:100180008DE090E0DF91CF911F910F91FF90EF9064
:10019000DF900895CF93DF93D92FC82F663429F5C8
:1001A0008091A2008A3309F580E258D18091A100A4
:1001B00055D18091A00052D18FEF50D195D188E2D6
:1001C0004DD18091A1004AD18091A00047D18FEFFD
:1001D00045D18AD18091A0009091A1000196909381
:1001E000A1008093A0002297F9F6DF91CF910895A6
:1001F000CFEDD0E0DEBFCDBFF894B898C09A000034
:10020000B099FFCF21D108D160E08BE090E068D1B8
:10021000B99AC19A6DD1813611F489E5B2C08134A1
:1002200089F466D199279093A1008093A000182F9C
:1002300000275ED19927082B192B1093A10000935A
:10024000A0003CC0823631F489E54ED180E04CD12B
:1002500080E497C0823471F44BD19927182F00277E
:1002600047D19927082B192B43D1682F912F802F25
:1002700024DF87C0873671F43BD19927182F0027D8
:1002800037D19927082B192B33D1682F912F802F25
:1002900081DFC0CF853631F48091A2008A3371F4BA
:1002A00013D10CC0853461F4BCD088E190E028E023
:1002B0000FB6F894A89581BD0FBE21BD8DE061C039
:1002C000803511F4E2D0FACF8C3411F4F4D0F6CFAB
:1002D000803711F483E555C0823711F48FEF51C098
:1002E0008C3611F405D1EACF843721F48AE3FCD0AF
:1002F00080E047C0883729F4FBD0823029F4C198C8
:10030000DDCF893719F4F4D0C19AD8CF843521F4E0
:10031000EFD08093A200D2CF833511F496DE7ACF4E
:10032000863521F480E3E0D082E32BC0833799F453
:100330008091A2008A3309F06DCF03E0015080E381
:100340008DD080E08BD0802F89D08FEF87D0CCD01C
:100350000023A1F75FCF8D3439F488B392E0892769
:1003600088BB84E7C1D0AACF8A3311F480E003C0F0
:100370008E3219F481E078DE4DCF8B3109F44ACF0B
:100380008FE3B2D047CFEF92FF920F931F93082FC6
:10039000192F802F912FAA2797FDA095BA2F682F8C
:1003A000792F8A2F9B2F09D117FF05C020E030E05D
:1003B00040E857E4A3D026E636E646E654E469D1A1
:1003C000E62EF72E082F192F20E030E040E85FE3FB
:1003D000FED088231CF481E090E017C020E03FEFBE
:1003E0004FE757E4912F802F7F2D6E2DF3D01816F5
:1003F0001CF480E090E009C0912F802F7F2D6E2D9E
:10040000BFD0B92FA82F972F862F0197F1F71F91F3
:100410000F91FF90EF900895C49885E190E0B3DFCD
:100420000895C49A85E190E0AEDF0895FADFF4DF25
:10043000089589E00000815087FFFCCF0895C79A96
:10044000F8DFC798F6DF0895BC9A0895C79A87B376
:10045000806A87BBF9DFBE98F2DF08950F931F9380
:10046000CF93082F10E0C0E8802F8C2311F0C59A9D
:1004700001C0C598B6991C0FE2DFC695A9F7812F78
:100480009927CF911F910F910895CF93DFDFCEDF92
:10049000C0E08CEAE3DF83E5E1DF8FEFDFDF833568
:1004A00011F4C1E401C0C2DF80E0D8DFCF5FC03407
:1004B00080F3CF910895BADF8FE597B3982397BB68
:1004C00098B3982398BB08958CEAC8DF80E8C6DF0C
:1004D00080E0C4DF80E0C2DF8AE090E054DF08956E
:1004E00089B988E18AB908955D9BFECF8CB90895DA
:1004F0005F9BFECF8CB1992708955058192EA6D036
:1005000001D08CC0BA176207730784079507B1F151
:1005100088F40EF410940B2EBA2FA02D062E622F05
:10052000202D072E732F302D082E842F402D092EBD
:10053000952F502DFF275523B9F0591B49F0573EF1
:1005400098F0469537952795A795F0405395C9F7AC
:1005500076F0BA0F621F731F841F30F4879577956A
:100560006795B795F040939517FA0F2E0895BF1B26
:10057000BB27BA0B620B730B840BF6CFDEF683C07E
:1005800097FB70D09F3738F0FEE9F91B982F872F23
:10059000762F6B2F05C074C09695879577956795D4
:1005A000F150D0F73EF490958095709561957F4F0E
:1005B0008F4F9F4F0895E89403C097FB0EF4F3DF2D
:1005C000B62F672F782F892F9EE9002427C00ED0E1
:1005D0005EF004C00BD026F001C008D019F020F462
:1005E0008FEF089580E0089581E0089597FB092E2C
:1005F000052600F868942DD0E89407FC07C0621720
:1006000073078407950721F008F4009407949894E1
:1006100008959A95BB0F661F771F881F1124992391
:10062000A1F08823B2F79F3F59F0BB0F48F421F4A3
:10063000002011F460FF04C06F5F7F4F8F4F9F4F0A
:10064000881F9795879597F908951AC0052E092652
:1006500007FA440F551F5F3F79F0AA27A51708F046
:1006600051E04795880F991F9F3F31F0BB27B9177D
:1006700008F091E0879508959F919F91112457C0AC
:1006800066277727882799270895592F482F372FCE
:10069000262FDCDF01D0C2CF992339F0552329F072
:1006A0009F575F57950F13F4CAF1EDCF91589F3FB5
:1006B000E1F3A62F00241124BB2766275527F8E075
:1006C000A69520F4020E131EB41F651F220F331FC0
:1006D000441F551FFA95A1F7F8E0E72F7727F8E0B8
:1006E000E69520F4130EB41F651F7A1F330F441FC5
:1006F000551FAA1FFA95A1F7F82F8827F69520F421
:10070000B40F651F7A1F8E1F440F551FAA1FEE1FBF
:10071000FF23A1F788231AF4939539F408C0000C3D
:10072000111CBB1F661F771F881F012808959FEFAC
:0407300080EC0895BC
:00000001FF
